:020000040000FA
:0600000026EF20F01200C3
:0614000026EF20F01200AF
:021408001200D0
:021418001200C0
:06142A0001006A40000011
:08143000C10000000B000000E8
:0814380065960F0139871FECD6
:1014400012F0040060EC16F0A5EC16F004000001A8
:10145000616B040E626F636B0001656B0001646B6E
:1014600061C066F062C067F063C068F00001A00E62
:10147000696F6A6B6B6B0001A00E6C6F6D6B6E6BAE
:101480000001726B61C073F062C074F063C075F0EC
:101490000001786B0001796B00017A6B00017B6BB6
:1014A0007C6B7D6B00016F6B706B716B0001816BEE
:1014B0000001826B0001976B986B996B00019A6B2E
:1014C0009B6B9C6B0001010E836F0001010E846F0A
:1014D0000001856B0001866B00019D6B9E6B9F6B0D
:1014E0000001876B0001886B0001A36BA46BA56BE7
:1014F0000001896B00018A6B00018D6B00017E6B1E
:101500007F6B806B0001010E8E6F00018F6B0001FD
:10151000A66BA76BA86B0001A96BAA6BAB6B000154
:10152000906B0001916B0001926B0001936B0001C5
:10153000946B0001956B0001AC6BAD6BAE6B000161
:10154000AF6BB06BB16B0001630E966F00018F51F2
:101550000BE180AE09D061C0A6F062C0A7F063C005
:10156000A8F00001010E8F6F80BE02D000018F6BCA
:1015700000018F051BE1A60EE96E000EEA6EEE502B
:101580000001615D006EEE5000016259016EEE5087
:1015900000016359026E140E001803E1015001E1CD
:1015A000025004E180AE02D00EEF00F0040057ECD0
:1015B00012F00400F2A425D0F294480ED76EE40E87
:1015C000D66E0001612B000E6223000E6323730EA2
:1015D000E96E000EEA6EEE500001615D006EEE50A5
:1015E00000016259016EEE5000016359026E080E4F
:1015F000005C000E0158000E025803E30001010ECA
:10160000786F0001790503E186EC1CF002D07CECD8
:101610001CF000017A5101E087D17E0EE96E000EC8
:10162000EA6EEE500001615D006EEE5000016259FD
:10163000016EEE5000016359026ED880010E005415
:10164000000E0154000E025405E30001790502E189
:1016500000018E6B00018E5106E10001795103E11A
:101660000001010E8E6F0001790556E17B0EE96ED7
:10167000000EEA6EEE500001615D006EEE5000015A
:101680006259016EEE5000016359026E040E005C57
:10169000000E0158000E02583FE300018E0535E1AF
:1016A0000001650517E10001656B61C069F062C06A
:1016B0006AF063C06BF00001A00E6C6F6D6B6E6B17
:1016C00089920001010E726F61C07BF062C07CF0F4
:1016D00063C07DF00001640517E10001646B61C027
:1016E0006CF062C06DF063C06EF00001A00E696F17
:1016F0006A6B6B6B89900001010E726F61C07BF0A9
:1017000062C07CF063C07DF007D000018E0504E16B
:101710000001646B0001656B6C0EE96E000EEA6EF1
:10172000EE500001615D006EEE5000016259016EE5
:10173000EE5000016359026EA40E005C000E0158C9
:10174000000E025801E2F0D0690EE96E000EEA6E5A
:10175000EE500001615D006EEE5000016259016EB5
:10176000EE5000016359026EA40E005C000E015899
:10177000000E025801E2D8D00001905102E0000EA4
:1017800001D0010E036E660EE96E000EEA6EEE5099
:101790000001615D006EEE5000016259016EEE5075
:1017A00000016359026E180E005C000E0158000E15
:1017B000025802E3000E01D0010E031044E00001C4
:1017C000655103E10001010E926F000192053AE1BB
:1017D000000165050CE1000190290001906F0001F6
:1017E000926B61C066F062C067F063C068F0030E80
:1017F0000001905D1FE161C069F062C06AF063C0E2
:101800006BF00001A00E6C6F6D6B6E6B8992000126
:10181000656B61C066F062C067F063C068F000018C
:10182000906B0001010E726F61C07BF062C07CF0B2
:1018300063C07DF00001640505E10001010E926FB7
:101840000001906B05D00001010E926F0001906BBA
:101850000001915102E0000E01D0010E036E660EF0
:10186000E96E000EEA6EEE500001615D006EEE5012
:1018700000016259016EEE5000016359026E180EAC
:10188000005C000E0158000E025802E3000E01D069
:10189000010E031044E00001645103E10001010E58
:1018A000936F000193053AE1000164050CE100012A
:1018B00091290001916F0001936B61C066F062C0D5
:1018C00067F063C068F0030E0001915D1FE161C025
:1018D0006CF062C06DF063C06EF00001A00E696F25
:1018E0006A6B6B6B89900001646B61C066F062C0CB
:1018F00067F063C068F00001916B0001010E726F28
:1019000061C07BF062C07CF063C07DF000016505C2
:1019100005E10001010E936F0001916B05D00001FC
:10192000010E936F0001916B81A2A0D16C0EE96E44
:10193000000EEA6EEE500001615D006EEE50000197
:101940006259016EEE5000016359026EA40E005CF4
:10195000000E0158000E025801E287D1690EE96EAF
:10196000000EEA6EEE500001615D006EEE50000167
:101970006259016EEE5000016359026EA40E005CC4
:10198000000E0158000E025801E26FD1AC0EE96E54
:10199000000EEA6EEE500001615D006EEE50000137
:1019A0006259016EEE5000016359026ED880040E38
:1019B0000054000E0154000E025401E356D181A4DC
:1019C00004D00001010E8B6F02D000018B6B81A649
:1019D00004D00001010E8C6F02D000018C6B00015D
:1019E00087510CE100018B5109E161C0A0F062C098
:1019F000A1F063C0A2F00001010E876F00018851C1
:101A00000CE100018C5109E161C0A3F062C0A4F0B7
:101A100063C0A5F00001010E886FA00EE96E000EF4
:101A2000EA6EEE500001615D006EEE5000016259F9
:101A3000016EEE5000016359026E010E001803E1C1
:101A4000015001E1025009E100018B5104E1000164
:101A5000010E896F02D00001876BA30EE96E000EA4
:101A6000EA6EEE500001615D006EEE5000016259B9
:101A7000016EEE5000016359026E010E001803E181
:101A8000015001E1025009E100018C5104E1000123
:101A9000010E8A6F02D00001886B6C0EE96E000E99
:101AA000EA6EEE500001615D006EEE500001625979
:101AB000016EEE5000016359026EA40E005C000E30
:101AC0000158000E025801E29AD0690EE96E000E2C
:101AD000EA6EEE500001615D006EEE500001625949
:101AE000016EEE5000016359026EA40E005C000E00
:101AF0000158000E025801E282D00001725101E04B
:101B00007ED07B0EE96E000EEA6EEE500001615D44
:101B1000006EEE5000016259016EEE5000016359F3
:101B2000026ED880080E0054000E0154000E0254BC
:101B300066E20001890530E1A00EE96E000EEA6E52
:101B4000EE500001615D006EEE5000016259016EC1
:101B5000EE5000016359026E020E005C000E015847
:101B6000000E025819E300018B0516E10001896B94
:101B70000001876B61C069F062C06AF063C06BF0FE
:101B80000001A00E6C6F6D6B6E6B89920001010EEF
:101B9000726F0001010E946F00018A0530E1A30EFF
:101BA000E96E000EEA6EEE500001615D006EEE50CF
:101BB00000016259016EEE5000016359026E020E7F
:101BC000005C000E0158000E025819E300018C055C
:101BD00016E100018A6B0001886B61C06CF062C085
:101BE0006DF063C06EF00001A00E696F6A6B6B6BE5
:101BF00089900001010E726F0001010E946FA00E1A
:101C0000E96E000EEA6EEE500001615D006EEE506E
:101C100000016259016EEE5000016359026E400EE0
:101C2000005C000E0158000E025804E30001896BAD
:101C30000001876BA30EE96E000EEA6EEE50000104
:101C4000615D006EEE5000016259016EEE500001C0
:101C50006359026E400E005C000E0158000E0258DF
:101C600004E300018A6B0001886B0FD000018D51E5
:101C70000CE081B40AD061C097F062C098F063C0F4
:101C800099F00001816B00018D6B81B42ED081B67B
:101C90002CD0899289900001726B0001A40E6C6FA8
:101CA0006D6B6E6B0001A40E696F6A6B6B6B61C02C
:101CB0007BF062C07CF063C07DF00001876B0001A7
:101CC000896B0001A06BA16BA26B0001886B000106
:101CD0008A6B0001A36BA46BA56B0001946B61C0C0
:101CE000ACF062C0ADF063C0AEF06C0EE96E000EF9
:101CF000EA6EEE500001615D006EEE500001625927
:101D0000016EEE5000016359026EA40E005C000EDD
:101D10000158000E02586CE3690EE96E000EEA6E7F
:101D2000EE500001615D006EEE5000016259016EDF
:101D3000EE5000016359026EA40E005C000E0158C3
:101D4000000E025855E30001835103E10001010E2A
:101D5000856F0001830512E1000185050FE1000197
:101D6000812B0001010E836F0001856B0001826BE6
:101D700061C09DF062C09EF063C09FF0030E000141
:101D8000815D08E361C097F062C098F063C099F08C
:101D90000001816B0001845103E10001010E866F97
:101DA0000001840512E1000186050FE10001822B8C
:101DB0000001010E846F0001866B0001816B61C020
:101DC0009DF062C09EF063C09FF0030E0001E76EBD
:101DD0008219E8AE02D0E73402D0E750825D08E312
:101DE00061C09AF062C09BF063C09CF00001826BFE
:101DF000690EE96E000EEA6EEE500001611908E10D
:101E0000EE500001621904E1EE500001631900E197
:101E10000DE100018D510AE061C097F062C098F0B9
:101E200063C099F00001816B00018D6B000181514D
:101E300000018225000826E29D0EE96E000EEA6E82
:101E4000EE500001615D006EEE5000016259016EBE
:101E5000EE5000016359026ED8800C0E0054000E43
:101E60000154000E02540EE20001816B0001826BEE
:101E70000001010E836F0001856B0001010E846F6C
:101E80000001866B970EE96E000EEA6EEE500001BF
:101E9000615D006EEE5000016259016EEE5000016E
:101EA0006359026ED880140E0054000E0154000EC7
:101EB000025405E3E9EC1EF000018D6B02D0DFEC6B
:101EC0001EF09A0EE96E000EEA6EEE500001615DA2
:101ED000006EEE5000016259016EEE500001635930
:101EE000026ED880140E0054000E0154000E0254ED
:101EF00006E3FDEC1EF00001010E8D6F02D0F3EC45
:101F00001EF0970EE96E000EEA6EEE500001615D64
:101F1000006EEE5000016259016EEE5000016359EF
:101F2000026ED880140E0054000E0154000E0254AC
:101F300018E30001815100018225000812E200012E
:101F4000976B986B996B0001816B0001826B0001AC
:101F5000010E836F0001856B0001010E846F00018B
:101F6000866B9A0EE96E000EEA6EEE500001615D1E
:101F7000006EEE5000016259016EEE50000163598F
:101F8000026ED880140E0054000E0154000E02544C
:101F900018E30001815100018225000812E20001CE
:101FA0009A6B9B6B9C6B0001816B0001826B000143
:101FB000010E836F0001856B0001010E846F00012B
:101FC000866B6F0EE96E000EEA6EEE500001615DE9
:101FD000006EEE5000016259016EEE50000163592F
:101FE000026ED880080E0054000E0154000E0254F8
:101FF00002E3899235D06C0EE96E000EEA6EEE5067
:102000000001615D006EEE5000016259016EEE50FC
:1020100000016359026EA00E005C000E0158000E14
:1020200002581EE26C0EE96E000EEA6EEE500001E0
:10203000615D006EEE5000016259016EEE500001CC
:102040006359026E020E001803E1015001E10250D3
:1020500007E00001720504E10001940501E18982B5
:102060006F0EE96E000EEA6EEE500001615D006ECB
:10207000EE5000016259016EEE5000016359026E8C
:10208000D880080E0054000E0154000E025402E3E2
:10209000899035D0690EE96E000EEA6EEE500001AF
:1020A000615D006EEE5000016259016EEE5000015C
:1020B0006359026EA00E005C000E0158000E02581B
:1020C0001EE2690EE96E000EEA6EEE500001615DDF
:1020D000006EEE5000016259016EEE50000163592E
:1020E000026E020E001803E1015001E1025007E008
:1020F0000001720504E10001940501E189806C0E84
:10210000E96E000EEA6EEE500001615D006EEE5069
:1021100000016259016EEE5000016359026EA00E7B
:10212000005C000E0158000E02581DE3690EE96EB6
:10213000000EEA6EEE500001615D006EEE5000018F
:102140006259016EEE5000016359026EA00E005CF0
:10215000000E0158000E025806E389928990000192
:10216000726B0001946B6C0EE96E000EEA6EEE501D
:102170000001615D006EEE5000016259016EEE508B
:1021800000016359026E020E001803E1015001E1E3
:10219000025004E10001965101E18992690EE96E55
:1021A000000EEA6EEE500001615D006EEE5000011F
:1021B0006259016EEE5000016359026E020E001862
:1021C00003E1015001E1025004E10001960501E143
:1021D00089906C0EE96E000EEA6EEE500001615DB2
:1021E000006EEE5000016259016EEE50000163591D
:1021F000026E280E001803E1015001E102501FE1B8
:10220000000196511CE1899289900001726B0001D6
:10221000A40E6C6F6D6B6E6B0001A40E696F6A6B20
:102220006B6B61C07BF062C07CF063C07DF000012D
:10223000946B61C0ACF062C0ADF063C0AEF0690EEB
:10224000E96E000EEA6EEE500001615D006EEE5028
:1022500000016259016EEE5000016359026E110EC9
:10226000001803E1015001E102501FE10001960551
:102270001CE1899289900001726B0001A40E6C6FC1
:102280006D6B6E6B0001A40E696F6A6B6B6B61C046
:102290007BF062C07CF063C07DF00001946B61C094
:1022A000ACF062C0ADF063C0AEF0730EE96E000E2C
:1022B000EA6EEE500001615D006EEE500001625961
:1022C000016EEE5000016359026ED880F00E00548A
:1022D000000E0154000E025401E3AED0898A010EB3
:1022E000E66E010EE66E2B0EE66EA1EC1EF0E552D8
:1022F000E552E552F19CF292F28804000300F2A24A
:1023000082D004000001010E956F010EE66E3DECD7
:102310001CF0E552E66A010EE66E2B0EE66EA1ECAD
:102320001EF0E552E552E552E66A010EE66E2C0E0D
:10233000E66EA1EC1EF0E552E552E552F298F292FB
:10234000899A0001B39F0001B39D0001B39BB3C004
:10235000E6FF0F0EE66ED8EC1CF0E552E5520E0ECD
:10236000E66E22EC1DF0E552E00B08E0B3C0E6FF9C
:102370000F0EE66ED8EC1CF0E552E5520001616BE1
:10238000040E626F636B0001666B676B686B000124
:10239000A00E696F6A6B6B6B0001A00E6C6F6D6BAA
:1023A0006E6B00017B6B7C6B7D6B00016F6B706BE8
:1023B000716B0001976B986B996B00019A6B9B6B2B
:1023C0009C6B00019D6B9E6B9F6B0001A36BA46BCC
:1023D000A56B00017E6B7F6B806B0001A66BA76B0A
:1023E000A86B0001A96BAA6BAB6B0001AC6BAD6B6A
:1023F000AE6B0001AF6BB06BB16B61C073F062C0CC
:1024000074F063C075F086EC1CF0050EE66EA4EC6B
:102410001CF0E5527CEC1CF080AE07D061C073F07C
:1024200062C074F063C075F007D00001950503E148
:102430000001956B01D062D7A6EF0AF012000F01E0
:102440001F0E486F0F011F0E496F9B8CFC0ED3149B
:102450000009D36E9482949C8B9C94948B940E016F
:10246000550EA76EAA0EA76EFF910C0EFB6F0A0EFB
:10247000D76F090ED36F550EA76EAA0EA76EFF81F8
:102480009290899092928992929489849296898668
:10249000929A899A929C898C928E9382F19E9490C2
:0E24A0008B8093849386938A949EC080120052
:0224AE00D8DB79
:1024B000030A01E14FD2010A01E13BD2030A09E01C
:1024C0000001725101E181D20001785101E17DD218
:1024D00067D2C60EE66E010EE66E0D0EE66E900E2B
:1024E000E66E7FEC1DF0E552E552E552E552E66AF4
:1024F000010EE66E2C0EE66EA1EC1EF0E552E552E2
:10250000E552C6C176F00001776BC6C177F0766BF5
:10251000000E7617FF0E7717E00E0101C7150001B8
:102520007625766F000E772176C000F0016E050EDD
:10253000D89001320032E804FBE100C076F001C01F
:1025400077F0280E0001001819E1020E771916E144
:10255000580E0101CF5D02E0000E01D0010E006EA9
:10256000180ECF5D02E0000E01D0010E001003E056
:102570000001836B03D00001010E836F280E000160
:10258000761919E1020E771916E1480E0101CF5DA7
:1025900002E0000E01D0010E006E080ECF5D02E0D9
:1025A000000E01D0010E001003E00001846B03D087
:1025B0000001010E846FC80E000176190DE1010EB5
:1025C00077190AE1040E0101D25D06E161C0AFF0A6
:1025D00062C0B0F063C0B1F0AF0EE96E000EEA6EFB
:1025E000EE500001615D026EEE506259036EEE50D6
:1025F0006359046ED880640E0254000E0354000E1A
:10260000045402E2000E01D0010E016E100E010111
:10261000CF15100802E0000E01D0010E006E680E0A
:102620000001761902E1030E771902E0000E01D0D5
:10263000010E0014011403E00001010E796F100E69
:102640000101CF15100802E1000E01D0010E006E4D
:10265000680E0001761902E1030E771902E0000E00
:1026600001D0010E001402E00001796BAF0EE96E9B
:10267000000EEA6EEE500001615D026EEE5062598E
:10268000036EEE506359046ED880640E0254000E3F
:102690000354000E045402E2000E01D0010E016E3C
:1026A0007F0E0101CB5D02E0000E01D0010E006E35
:1026B000680E0001761902E1030E771902E0000EA0
:1026C00001D0010E0014011403E00001010E796F26
:1026D000AF0EE96E000EEA6EEE500001615D006E15
:1026E000EE506259016EEE506359026ED880640E4E
:1026F0000054000E0154000E025402E20001796BF6
:102700000001880E761915E1775113E1060E0101DB
:10271000CD15060804E10001010E7A6F0AD0000110
:102720007A0506E161C07EF062C07FF063C080F090
:102730007A6B00017A5101E0E3D00001880E76192E
:102740000BE1775109E10001720506E10101060E76
:10275000CD6F0001010E946FC80E0001761901E0E3
:102760007ED0010E771901E07AD07B0EE96E000E63
:10277000EA6EEE500001615D006EEE506259016E2E
:10278000EE506359026E040E005C000E0158000EFC
:10279000025865E3020E0101D25D28E16C0EE96E7C
:1027A000000EEA6EEE500001615D006EEE5062595F
:1027B000016EEE506359026EA00E005C000E0158CF
:1027C000000E025813E2899289900001726B000199
:1027D000A40E6C6F6D6B6E6B0001696F6A6B6B6B37
:1027E00061C07BF062C07CF063C07DF00101CD056B
:1027F00002E0000E01D0010E006ED20502E0000ED4
:1028000001D0010E00102BE0690EE96E000EEA6E99
:10281000EE500001615D006EEE506259016EEE50A7
:102820006359026EA00E005C000E0158000E0258A3
:1028300016E20001905113E1899289900001726BB8
:102840000001A40E6C6F6D6B6E6B0001696F6A6B9B
:102850006B6B61C07BF062C07CF063C07DF0C80E22
:10286000000176194DE1010E77194AE17B0EE96E00
:10287000000EEA6EEE500001615D006EEE5062598E
:10288000016EEE506359026E040E005C000E01589A
:10289000000E025835E3020E0101D25D05E1000190
:1028A000010E646F0001656B0101D20505E10001B5
:1028B000010E656F0001646B0101CD0505E10001AA
:1028C000010E656F0001646B0101CD0519E0110E69
:1028D000E76ED219E8AE02D0E73402D0E750D25DFD
:1028E0000FE3150EE76ED219E8AE02D0D23503D051
:1028F000E750D880D25504E30001646B0001656B9A
:10290000C60EE66E010EE66E0D0EE66EE66876EC1D
:102910001BF0E552E552E552E55261C073F062C02A
:1029200074F063C075F0E66A2D0EE66ED8EC1CF00C
:1029300034D0C60EE66E010EE66E0D0EE66E940EF7
:10294000E66E7FEC1DF0E552E552E552E552E66A8F
:10295000020E10D0C60EE66E010EE66E0D0EE66E8D
:10296000900EE66E7FEC1DF0E552E552E552E55221
:10297000E66A010EE66E2C0EE66EA1EC1EF0E55244
:10298000E552E552C60EE66E010EE66E0D0EE66EDF
:10299000E66876EC1BF0E552E552E552E55215D0BB
:1029A000C60EE66E010EE66E0D0EE66EE66876EC7D
:1029B0001BF0E552E552E552E55261C073F062C08A
:1029C00074F063C075F00001786B1AD9030A01E155
:1029D000F1D0010A01E1DDD0030A01E01200A60EE8
:1029E000E66E010EE66E0D0EE66E900EE66E39ECAA
:1029F0001BF0E552E552E552E552E66A010EE66E3D
:102A00002C0EE66E5BEC1CF0E552E552E552A6C1D9
:102A100076F00001776BA6C177F0766B000E761723
:102A2000FF0E7717E00E0101A71500017625766FDE
:102A3000000E772176C000F0016E050ED8900132AD
:102A40000032E804FBE100C076F001C077F000013D
:102A50007A5131E1100E0101B2150001C16F3F0E34
:102A60000001761928E1040E771925E100017205AD
:102A700022E1100E0001C15D1EE16F0EE96E000E35
:102A8000EA6EEE500001615D006EEE506259016E1B
:102A9000EE506359026ED880100E0054000E01549F
:102AA000000E025408E261C06FF062C070F063C0B3
:102AB00071F0899289903F0E0001761901E092D061
:102AC000040E771901E08ED0B2C196F0690EE96E5E
:102AD000000EEA6EEE500001615D006EEE5062592C
:102AE000016EEE506359026EA00E005C000E01589C
:102AF000000E02581CE20001965119E1899289905A
:102B00000001726B0001A40E6C6F6D6B6E6B0001A7
:102B1000696F6A6B6B6B61C07BF062C07CF063C0F5
:102B20007DF00001946B0001AF6FB06BB16B6C0E68
:102B3000E96E000EEA6EEE500001615D006EEE502F
:102B40006259016EEE506359026EA00E005C000ED9
:102B50000158000E025846E20001960543E18992B1
:102B600089900001726B0001A40E6C6F6D6B6E6B2F
:102B70000001696F6A6B6B6B61C07BF062C07CF0B7
:102B800063C07DF00001946B0001AF6FB06BB16B5F
:102B900029D0A60EE66E010EE66E0D0EE66E940EC0
:102BA000E66E39EC1BF0E552E552E552E552E66A75
:102BB000020E10D0A60EE66E010EE66E0D0EE66E4B
:102BC000900EE66E39EC1BF0E552E552E552E55207
:102BD000E66A010EE66E2C0EE66E5BEC1CF0E5522A
:102BE000E552E552A60EE66E010EE66E0D0EE66E9D
:102BF000E668BCEC1DF0E552E552E552E5521200E4
:102C0000D9CFE6FFE1CFD9FFE6520101FD93FD9553
:102C100028EC1CF0DF6EDFA00CD00101FD51060B8B
:102C2000E8420109030BF36EF346F90EFD15F310AC
:102C3000FD6FDFA20CD00101FD51060BE842020935
:102C4000030BF36EF346F90EFD15F310FD6F010152
:102C5000FD51060BE842E552E552E7CFD9FF1200DD
:102C6000D9CFE6FFE1CFD9FFE6520101FE93FE95F1
:102C70006EEC1EF0DF6EDFA00CD00101FE51060BE2
:102C8000E8420109030BF36EF346F90EFE15F3104B
:102C9000FE6FDFA20CD00101FE51060BE8420209D3
:102CA000030BF36EF346F90EFE15F310FE6F0101F0
:102CB000FE51060BE842E552E552E7CFD9FF12007C
:102CC000D9CFE6FFE1CFD9FFE65289849294E66A34
:102CD000E66A010EE66E81EC1FF0E552E552E55220
:102CE000938A9398DF6ADFCF00F0400EE76E0018FA
:102CF000E8AE02D0E73402D0E750005C16E2DFCF46
:102D0000E9FFEA6AE9BEEA68050EE926010EEA2251
:102D1000EF6ADFCFE9FFEA6AE9BEEA68450EE92615
:102D2000010EEA22EF6ADF2ADED7480ED76EE40EE4
:102D3000D66ED596D584D592D580D59AD59C49D8CE
:102D4000E552E552E7CFD9FF1200D9CFE6FFE1CF38
:102D5000D9FFE65289869296E66AE66A010EE66E29
:102D600056EC1FF0E552E552E552DF6ADFCF00F086
:102D7000400EE76E0018E8AE02D0E73402D0E7500C
:102D8000005C16E2DFCFE9FFEA6AE9BEEA68050EF9
:102D9000E926010EEA22EF6ADFCFE9FFEA6AE9BE1F
:102DA000EA68450EE926010EEA22EF6ADF2ADED73D
:102DB000480ED76EE40ED66ED596D584D592D580C2
:102DC000D59A0101FD9D3DD9E552E552E7CFD9FFE6
:102DD0001200D9CFE6FFE1CFD9FFE6527BEC1AF023
:102DE000DF6ADF50006E016AD890015004E6FA0EE7
:102DF000005C000E015802E2DF2AF3D70001B38F16
:102E0000B39DB39BB397B399B395B3C0E6FF0F0ED1
:102E1000E66E92EC1AF0E552E5520E0EE66EDCEC30
:102E20001AF0E552E00B800808E0B3C0E6FF0F0E91
:102E3000E66E92EC1AF0E552E5520101866B876B63
:102E4000886B896B860EE66E010EE66E040EE66EEA
:102E5000200EE66EADEC1AF0E552E552E552E55271
:102E6000860EE66E010EE66E040EE66E240EE66E2B
:102E7000ADEC1AF0E552E552E552E552E66A010E74
:102E8000E66E92EC1AF0E552E552E66A050EE66E41
:102E900092EC1AF0E552E552080EE66E090EE66E67
:102EA00092EC1AF0E552E552080EE66E110EE66E4F
:102EB00092EC1AF0E552E552080EE66E150EE66E3B
:102EC00092EC1AF0E552E552080EE66E190EE66E27
:102ED00092EC1AF0E552E5520101A30E866F090E3D
:102EE000876F120E886F340E896F040E8A6F8B6B9A
:102EF000010E8C6F020E8D6F030E8E6F040E8F6F9E
:102F0000050E906F060E916F070E926F860EE66E9D
:102F1000010EE66E0D0EE66E400EE66E76EC1BF0D0
:102F2000E552E552E552E5520101220E866F876BAC
:102F3000640E886F680E896F020E8A6F8B6B110E9C
:102F40008C6F220E8D6F330E8E6F440E8F6F550E69
:102F5000906F660E916F770E926F860EE66E010E81
:102F6000E66E0D0EE66E420EE66E76EC1BF0E55256
:102F7000E552E552E5520101AA0E866F030E876FF6
:102F8000330E886F896F080E8A6FAA0E8B6FBB0E87
:102F90008C6FCC0E8D6FDD0E8E6FEE0E8F6F906985
:102FA0000A0E916F0B0E926F860EE66E010EE66EA4
:102FB0000D0EE66E440EE66E76EC1BF0E552E55221
:102FC000E552E5520001B68F070EE66E74D9E55260
:102FD0000001B39FB39DB39BB3C0E6FF0F0EE66E37
:102FE00092EC1AF0E552E5520101856B0E0EE66E89
:102FF000DCEC1AF0E552E00B08E0B3C0E6FF0F0E80
:10300000E66E92EC1AF0E552E5520001BA85BA91EB
:10301000BA87BA93BAC0E6FF0C0EE66E92EC1AF0CD
:10302000E552E552E668300EE66E0C0EE66E5BEC9D
:103030001CF0E552E552E552E552E552E7CFD9FFE3
:103040001200D9CFE6FFE1CFD9FFE652C1EC1CF068
:10305000DF6ADF50006E016AD890015004E6FA0E74
:10306000005C000E015802E2DF2AF3D70001B38FA3
:10307000B39DB39BB397B399B385B393B391B3C0E7
:10308000E6FF0F0EE66ED8EC1CF0E552E5520E0E90
:10309000E66E22EC1DF0E552E00B800808E0B3C0BC
:1030A000E6FF0F0EE66ED8EC1CF0E552E55201018A
:1030B000866B876B886B896B860EE66E010EE66EFB
:1030C000040EE66E200EE66EF3EC1CF0E552E552BF
:1030D000E552E552860EE66E010EE66E040EE66ED1
:1030E000240EE66EF3EC1CF0E552E552E552E55293
:1030F000E66A010EE66ED8EC1CF0E552E552E66A8F
:10310000050EE66ED8EC1CF0E552E552080EE66EB0
:10311000090EE66ED8EC1CF0E552E552080EE66E9C
:10312000110EE66ED8EC1CF0E552E552080EE66E84
:10313000150EE66ED8EC1CF0E552E552080EE66E70
:10314000190EE66ED8EC1CF0E552E5520101A30E13
:10315000866F090E876F120E886F340E896F040E0A
:103160008A6F8B6B010E8C6F020E8D6F030E8E6F4C
:10317000040E8F6F050E906F060E916F070E926F03
:10318000860EE66E010EE66E0D0EE66E400EE66EE3
:10319000BCEC1DF0E552E552E552E5520101220E6C
:1031A000866F876B640E886F680E896F020E8A6F58
:1031B0008B6B110E8C6F220E8D6F330E8E6F440E43
:1031C0008F6F550E906F660E916F770E926F860E11
:1031D000E66E010EE66E0D0EE66E420EE66EBCEC7D
:1031E0001DF0E552E552E552E5520101AA0E866F47
:1031F000030E876F330E886F896F080E8A6FAA0ED1
:103200008B6FBB0E8C6FCC0E8D6FDD0E8E6FEE0E46
:103210008F6F90690A0E916F0B0E926F860EE66E9D
:10322000010EE66E0D0EE66E440EE66EBCEC1DF071
:10323000E552E552E552E5520001B68F070EE66E03
:10324000C9D8E5520001B39FB39DB39BB3C0E6FF5D
:103250000F0EE66ED8EC1CF0E552E5520101856BCD
:103260000E0EE66E22EC1DF0E552E00B08E0B3C056
:10327000E6FF0F0EE66ED8EC1CF0E552E5520001B9
:10328000BA85BA91BA87BA93BAC0E6FF0C0EE66E59
:10329000D8EC1CF0E552E552E66A300EE66E0C0EF4
:1032A000E66EA1EC1EF0E552E552E552E552E5521C
:1032B000E7CFD9FF1200D9CFE6FFE1CFD9FF040E47
:1032C000E1260001B38FB39DB39BB3C0E6FF0F0EA1
:1032D000E66E92EC1AF0E552E5520E0EE66EDCEC6C
:1032E0001AF0E552E00B800808E0B3C0E6FF0F0ECD
:1032F000E66E92EC1AF0E552E5520001B46B000163
:10330000B56B0001B66B0001B49FB49D0001B5958B
:10331000B583B591B59BB589B5970001B695B683D0
:10332000B6910001B58FB58DFE0EDB5015E0010A98
:103330000EE0020A07E0040A13E1C00E0001B41512
:10334000070F0DD0C00E0001B415030F08D0C00E3A
:103350000001B415010F03D0C00E0001B415B46F05
:10336000B6C086F1B5C087F1B4C088F1860EE66EAE
:10337000010EE66E030EE66E280EE66EADEC1AF058
:10338000E552E552E552E5520001B39FB39DB39B70
:10339000B3C0E6FF0F0EE66E92EC1AF0E552E5526E
:1033A0000E0EE66EDCEC1AF0E552E00B800808E049
:1033B000B3C0E6FF0F0EE66E92EC1AF0E552E5524E
:1033C000040EE15C02E2E16AE552E16EE552E7CF0C
:1033D000D9FF1200D9CFE6FFE1CFD9FF040EE126D5
:1033E0000001B38FB39DB39BB3C0E6FF0F0EE66E33
:1033F000D8EC1CF0E552E5520E0EE66E22EC1DF004
:10340000E552E00B800808E0B3C0E6FF0F0EE66E61
:10341000D8EC1CF0E552E5520001B46B0001B56B2D
:103420000001B66B0001B49FB49D0001B595B58352
:10343000B591B59BB589B5970001B695B683B691A0
:103440000001B58FB58DFE0EDB5015E0010A0EE0D0
:10345000020A07E0040A13E1C00E0001B415070FC9
:103460000DD0C00E0001B415030F08D0C00E00012E
:10347000B415010F03D0C00E0001B415B46FB6C06F
:1034800086F1B5C087F1B4C088F1860EE66E010EF4
:10349000E66E030EE66E280EE66EF3EC1CF0E552C7
:1034A000E552E552E5520001B39FB39DB39BB3C013
:1034B000E6FF0F0EE66ED8EC1CF0E552E5520E0E5C
:1034C000E66E22EC1DF0E552E00B800808E0B3C088
:1034D000E6FF0F0EE66ED8EC1CF0E552E552040E46
:1034E000E15C02E2E16AE552E16EE552E7CFD9FF25
:0634F000120012001200A0
:0A34F6008994C00EE66ECAEC1FF0C8
:10350000E55289840001D66BD651006E016AD890CD
:10351000015004E6FF0E005C000E015802E2D62BBB
:10352000F3D71200D9CFE6FFE1CFD9FF8994020E7D
:10353000E66ECAEC1FF0E552FE0EDBCFE6FFCAECEA
:103540001FF0E552FD0EDBCFE6FFCAEC1FF0E5529F
:103550008984E552E7CFD9FF1200D9CFE6FFE1CF4A
:10356000D9FFE6528994020EE66ECAEC1FF0E552CE
:10357000FE0EDBCFE6FFCAEC1FF0E552DF6AFD0E60
:10358000DB50DF5C13E2DF50E76EFB0EDBCFE9FFC1
:10359000FC0EDBCFEAFFE750E926000EEA22EF50EF
:1035A000E66ECAEC1FF0E552DF2AE9D78984E552BE
:1035B000E552E7CFD9FF1200D9CFE6FFE1CFD9FF1F
:1035C000E6528994030EE66ECAEC1FF0E552FE0E39
:1035D000DBCFE6FFCAEC1FF0E552FFEC1FF0DF6E19
:1035E0008984DF50E552E552E7CFD9FF1200D9CFE9
:1035F000E6FFE1CFD9FFE6528994030EE66ECAECEE
:103600001FF0E552FE0EDBCFE6FFCAEC1FF0E552DD
:10361000DF6AFD0EDB50DF5C14E2FFEC1FF0E66EAC
:10362000DF50E76EFB0EDBCFE9FFFC0EDBCFEAFFDE
:10363000E750E926000EEA22E552E750EF6EDF2A56
:10364000E8D7FFEC1FF0E66EDF50E76EFB0EDBCF36
:10365000E9FFFC0EDBCFEAFFE750E926000EEA2285
:10366000E552E750EF6E8984E552E552E7CFD9FF86
:103670001200D9CFE6FFE1CFD9FFE6528994FE0EC2
:10368000DBCFE6FFCAEC1FF0E552DF6AFD0EDB5030
:10369000DF5C14E2FFEC1FF0E66EDF50E76EFB0E1E
:1036A000DBCFE9FFFC0EDBCFEAFFE750E926000E97
:1036B000EA22E552E750EF6EDF2AE8D7FFEC1FF071
:1036C000E66EDF50E76EFB0EDBCFE9FFFC0EDBCFD3
:1036D000EAFFE750E926000EEA22E552E750EF6ED6
:1036E0008984E552E552E7CFD9FF1200D9CFE6FF32
:1036F000E1CFD9FF030EE126FE0EDB50FF0838E1D3
:10370000A7D8DF6EDFBC07D0440EF36EFE0EF3CFFA
:10371000DBFF840E29D0DFB807D0420EF36EFE0E19
:10372000F3CFDBFF820E20D0DFA418D0540EDF14BD
:103730001FE0E66A300EE66EF5DEE552E552000166
:10374000D66BD651006E016AD890015004E6FF0E88
:10375000005C000E015802E2D62BF3D7400EF36E48
:10376000FE0EF3CFDBFF810EF36E020EF3CFDBFF15
:103770008994FE0EDBCFE6FFCAEC1FF0E552DF6A4C
:10378000FD0EDB50DF5C13E2DF50E76EFB0EDBCF9C
:10379000E9FFFC0EDBCFEAFFE750E926000EEA2244
:1037A000EF50E66ECAEC1FF0E552DF2AE9D78984B4
:1037B000020EDBCFE6FF0FD8E552FE0EDB50006EA7
:1037C000030EE15C02E2E16AE552E16E0050E5526F
:1037D000E7CFD9FF1200D9CFE6FFE1CFD9FFE652FC
:1037E000FE0EDBA00ED0E66A300EE66E9BDEE552E2
:1037F000E5528994FE0EDBCFE6FFCAEC1FF0E552DE
:103800008984FE0EDBA20ED0E66A400EE66E8ADEEA
:10381000E552E5528994FE0EDBCFE6FFCAEC1FF0BD
:10382000E5528984FE0EDBA40ED0E66A500EE66EE9
:1038300079DEE552E5528994FE0EDBCFE6FFCAEC55
:103840001FF0E5528984E552E552E7CFD9FF120017
:10385000D9CFE6FFE1CFD9FFE6528994A00EE66EFC
:10386000CAEC1FF0E552FFEC1FF0DF6E8984DF50D9
:10387000E552E552E7CFD9FF1200D9CFE6FFE1CFFD
:10388000D9FFE652CF0ECF6E2B0ECE6ECD80DF6A03
:10389000FE0EDB50DF5C09E29EA0FED79E90CF0EAD
:1038A000CF6E2B0ECE6EDF2AF3D7CD90E552E552C8
:1038B000E7CFD9FF1200D9CFE6FFE1CFD9FF899436
:1038C000050EE66ECAEC1FF0E552FE0EDBCFE6FFFA
:1038D000CAEC1FF0E552FD0EDBCFE6FFCAEC1FF08D
:1038E000E552FC0EDBCFE6FFCAEC1FF0E5528984FF
:1038F000E552E7CFD9FF1200E668100EE66E0C0E17
:10390000E66ED9DFE552E552E5521200E66A100E86
:10391000E66E0C0EE66ECFDFE552E552E552120080
:10392000E668200EE66E0C0EE66EC5DFE552E55247
:10393000E5521200E66A200EE66E0C0EE66EBBDF64
:10394000E552E552E5521200D9CFE6FFE1CFD9FFAB
:10395000E652350ECF6ECE6ACD80DF6AFE0EDB50AA
:10396000DF5C09E29EA0FED79E90CF0ECF6E2B0E9D
:10397000CE6EDF2AF3D7CD90E552E552E7CFD9FFDF
:02398000120033
:0E3982008996C00EE66EACEC1FF0E552898609
:103990000001D76BD751006E016AD890015004E640
:1039A000FF0E005C000E015802E2D72BF3D7120085
:1039B000D9CFE6FFE1CFD9FF8996020EE66EACECD7
:1039C0001FF0E552FE0EDBCFE6FFACEC1FF0E55238
:1039D000FD0EDBCFE6FFACEC1FF0E5528986E55229
:1039E000E7CFD9FF1200D9CFE6FFE1CFD9FFE652EA
:1039F0008996020EE66EACEC1FF0E552FE0EDBCFB0
:103A0000E6FFACEC1FF0E552DF6AFD0EDB50DF5C39
:103A100013E2DF50E76EFB0EDBCFE9FFFC0EDBCFDE
:103A2000EAFFE750E926000EEA22EF50E66EACEC22
:103A30001FF0E552DF2AE9D78986E552E552E7CF44
:103A4000D9FF1200D9CFE6FFE1CFD9FFE652899620
:103A5000030EE66EACEC1FF0E552FE0EDBCFE6FF88
:103A6000ACEC1FF0E552E8EC1FF0DF6E8986DF500A
:103A7000E552E552E7CFD9FF1200D9CFE6FFE1CFFB
:103A8000D9FFE6528996030EE66EACEC1FF0E552C4
:103A9000FE0EDBCFE6FFACEC1FF0E552DF6AFD0E59
:103AA000DB50DF5C14E2E8EC1FF0E66EDF50E76EFF
:103AB000FB0EDBCFE9FFFC0EDBCFEAFFE750E92688
:103AC000000EEA22E552E750EF6EDF2AE8D7E8EC75
:103AD0001FF0E66EDF50E76EFB0EDBCFE9FFFC0E5A
:103AE000DBCFEAFFE750E926000EEA22E552E75075
:103AF000EF6E8986E552E552E7CFD9FF1200D9CFA4
:103B0000E6FFE1CFD9FFE6528996FE0EDBCFE6FF56
:103B1000ACEC1FF0E552DF6AFD0EDB50DF5C14E217
:103B2000E8EC1FF0E66EDF50E76EFB0EDBCFE9FF3F
:103B3000FC0EDBCFEAFFE750E926000EEA22E55251
:103B4000E750EF6EDF2AE8D7E8EC1FF0E66EDF50B3
:103B5000E76EFB0EDBCFE9FFFC0EDBCFEAFFE750A1
:103B6000E926000EEA22E552E750EF6E8986E5521B
:103B7000E552E7CFD9FF1200D9CFE6FFE1CFD9FF59
:103B8000030EE126FE0EDB50FF0838E1A7D8DF6EFA
:103B9000DFBC07D0440EF36EFE0EF3CFDBFF840EC6
:103BA00029D0DFB807D0420EF36EFE0EF3CFDBFF55
:103BB000820E20D0DFA418D0540EDF141FE0E66A76
:103BC000300EE66EF5DEE552E5520001D76BD751B7
:103BD000006E016AD890015004E6FF0E005C000EF2
:103BE000015802E2D72BF3D7400EF36EFE0EF3CF4F
:103BF000DBFF810EF36E020EF3CFDBFF8996FE0E24
:103C0000DBCFE6FFACEC1FF0E552DF6AFD0EDB50C8
:103C1000DF5C13E2DF50E76EFB0EDBCFE9FFFC0E4B
:103C2000DBCFEAFFE750E926000EEA22EF50E66E0E
:103C3000ACEC1FF0E552DF2AE9D78986020EDBCF14
:103C4000E6FF0FD8E552FE0EDB50006E030EE15C7E
:103C500002E2E16AE552E16E0050E552E7CFD9FF9A
:103C60001200D9CFE6FFE1CFD9FFE652FE0EDBA06E
:103C70000ED0E66A300EE66E9BDEE552E55289967E
:103C8000FE0EDBCFE6FFACEC1FF0E5528986FE0EA0
:103C9000DBA20ED0E66A400EE66E8ADEE552E55201
:103CA0008996FE0EDBCFE6FFACEC1FF0E55289866D
:103CB000FE0EDBA40ED0E66A500EE66E79DEE5520B
:103CC000E5528996FE0EDBCFE6FFACEC1FF0E55225
:103CD0008986E552E552E7CFD9FF1200D9CFE6FF3A
:103CE000E1CFD9FFE6528996A00EE66EACEC1FF04C
:103CF000E552E8EC1FF0DF6E8986DF50E552E552B1
:103D0000E7CFD9FF1200D9CFE6FFE1CFD9FFE652C6
:103D1000CF0ECF6E2B0ECE6ECD80DF6AFE0EDB5047
:103D2000DF5C09E29EA0FED79E90CF0ECF6E2B0ED9
:103D3000CE6EDF2AF3D7CD90E552E552E7CFD9FF1B
:103D40001200D9CFE6FFE1CFD9FF8996050EE66EC6
:103D5000ACEC1FF0E552FE0EDBCFE6FFACEC1FF043
:103D6000E552FD0EDBCFE6FFACEC1FF0E552FC0E9A
:103D7000DBCFE6FFACEC1FF0E5528986E552E7CFDA
:103D8000D9FF1200D9CFE6FFE1CFD9FFE652350EB9
:103D9000CF6ECE6ACD80DF6AFE0EDB50DF5C09E2BB
:103DA0009EA0FED79E90CF0ECF6E2B0ECE6EDF2A3A
:103DB000F3D7CD90E552E552E7CFD9FF1200E66A7E
:103DC000100EE66E0C0EE66EBCDFE552E552E552D3
:103DD0001200E668100EE66E0C0EE66EB2DFE552DB
:103DE000E552E5521200E66A200EE66E0C0EE66E13
:103DF000A8DFE552E552E5521200E668200EE66EB5
:0E3E00000C0EE66E9EDFE552E552E552120012
:023E0E002A0E7A
:103E1000F66E140EF76E000EF86E00010900F550F4
:103E2000D16F0900F550D26F03E1D16701D03DD0C9
:103E30000900F550CC6F0900F550CD6F0900F55021
:103E4000CE6F09000900F550E96E0900F550EA6EE1
:103E5000090009000900F550CF6F0900F550D06F37
:103E600009000900F6CFD3F0F7CFD4F0F8CFD5F0A2
:103E7000CCC0F6FFCDC0F7FFCEC0F8FF0001CF5396
:103E800002E1D05307E00900F550EE6ECF07F8E2EB
:103E9000D007F9D7D3C0F6FFD4C0F7FFD5C0F8FFDD
:0C3EA0000001D107000ED25BBFD712005A
:043EAC00D9CFE6FF85
:103EB000DACFE6FFE1CFD9FFE2CFDAFF3F0E73168C
:103EC000726AFD0EDB507212FB0EDB507312FC0E99
:103ED000DB50030A09E0010A04E0020A06E1738CE0
:103EE00004D0738C728801D07288FD0EDB50050AF5
:103EF00001E0010A728AE552E5CFDAFFE7CFD9FF88
:023F00001200AD
:0E3F0200D9CFE6FFDACFE6FFE1CFD9FFE2CF5D
:103F1000DAFF3F0EC716C66AFD0EDB50C612FB0E57
:103F2000DB50C712FC0EDB50030A09E0010A04E073
:103F3000020A06E1C78C04D0C78CC68801D0C688A7
:103F4000FD0EDB50050A01E0010AC68AE552E5CF05
:083F5000DAFFE7CFD9FF1200F0
:083F5800D9CFE6FFDACFE6FF46
:103F6000E1CFD9FFE2CFDAFFE6527550DF6EA49EB3
:103F7000729EFD0EDB50756E72AE02D0FF0E03D046
:103F8000A4AEFED7000EE552E552E5CFDAFFE7CF4B
:043F9000D9FF120043
:0C3F9400D9CFE6FFDACFE6FFE1CFD9FF7E
:103FA000E2CFDAFFE652C950DF6E9E96C69EFD0E46
:103FB000DB50C96EC6AE02D0FF0E03D09EA6FED760
:103FC000000EE552E552E5CFDAFFE7CFD9FF120048
:103FD000D9CFE6FFDACFE6FFE1CFD9FFE2CFDAFFB4
:103FE000E6527550DF6EA49E756AA4AEFED775507A
:0E3FF000E552E552E5CFDAFFE7CFD9FF120028
:023FFE00D9CF19
:10400000E6FFDACFE6FFE1CFD9FFE2CFDAFFE652F3
:10401000C950DF6E9E96C96A9EA6FED7C950E5526A
:0C402000E552E5CFDAFFE7CFD9FF120030
:04402C00C00EF36E61
:1040300000EE00F00E0E01D81200EA6002D0EE6A27
:0C404000FCD7F350E9601200EE6AFCD7D8
:04404C001DEE00F075
:104050002DEE00F0F86A069C07EC1FF034EC20F01F
:084060001CEC0AF0FBD7120072
:02406800120044
:06406A000001F00000005F
:054070000080000100CA
:017FF8008CFC
:017FF900F790
:017FFA000284
:017FFB00F88D
:017FFC00F193
:017FFD00F88B
:017FFE00DFA3
:017FFF00F190
:00000001FF
